:100000000C947F010C94A7010C94A7010C94A701F8
:100010000C94A7010C94A7010C94A7010C94A701C0
:100020000C94A7010C94A7010C94AB0B0C94770AC9
:100030000C94A7010C94A7010C94A7010C94A701A0
:100040000C94A7010C94A7010C94A7010C94A70190
:100050000C94A7010C94A7010C94A7010C940C0D0F
:100060000C94A7010C94A7010C94A7010C94A70170
:100070000C94A7010C94A7010C94A7010C94A70160
:100080000C94A7010C94A7010C94A7010C94A70150
:100090000C94A7010C94A7010C94A7010C94A70140
:1000A0000C94A7010C94A7010C94A701DF05E405AB
:1000B000E905F305FD05470647064706070611064D
:1000C0001B062506320647063A0668066B065A06E0
:1000D0005E0664068C068C068C066F067306770631
:1000E0007D0681068C0687060000000200090F00CD
:1000F00000030401000C00000000000000000000EC
:1001000000000000000004080201104080401020A0
:1001100040804080080204018040201002011080CD
:1001200010204040040404040403040502020202F7
:100130000403020202020606060606060404020280
:100140000204000000002300260029002C002F00DC
:1001500000000000250028002B002E0031000000C8
:100160000000240027002A002D003000080B0002A8
:10017000020201000904000001020200000524003F
:1001800010010524010101042402060524060001D2
:100190000705810310004009040100020A00000065
:1001A000070502024000000705830240000000C16D
:1001B0008081C1120100020200004041233680000C
:1001C000010102000112010002000000404123363B
:1001D0008000010102000141726475696E6F204C5C
:1001E0004C430041726475696E6F204C656F6E619F
:1001F00072646F00040309040000000000000000A6
:100200002A2B280000000000000000000000000071
:1002100000000000000000002C9EB4A0A1A2A434A5
:10022000A6A7A5AE362D3738271E1F20212223244E
:100230002526B333B62EB7B89F8485868788898AEA
:100240008B8C8D8E8F909192939495969798999A86
:100250009B9C9D2F3130A3AD350405060708090A84
:100260000B0C0D0E0F101112131415161718191A66
:100270001B1C1DAFB1B0B500090402000103000052
:1002800000092101010001226500070584034000E7
:100290000105010902A1010901A100850105091952
:1002A000012903150025019503750181029501754A
:1002B00005810305010930093109381581257F754C
:1002C0000895038106C0C005010906A10185020544
:1002D0000719E029E71500250175019508810295A8
:1002E0000175088103950675081500256505071930
:1002F0000029658100C07702E8072D0F7D021124D7
:100300001FBECFEFDAE0DEBFCDBF11E0A0E0B1E06D
:10031000ECE0F3E202C005900D92AE35B107D9F7DB
:1003200021E0AEE5B1E001C01D92A43FB207E1F7C4
:1003300012E0CCEFD2E004C02297FE010E943D0FF4
:10034000C63FD107C9F70E9406080C9479110C9496
:10035000000060E080911E010E948D0660E08091A7
:1003600018010E948D0680917C0190917D01823060
:10037000910531F460E0809116010E948D0612C053
:1003800061E0019731F4809116010E948D0660E0D2
:1003900005C0809116010E948D0661E080911601D2
:1003A0000E94C60661E080911C010E948D0661E0FA
:1003B00080911A010E948D0661E0809114010E94D3
:1003C0008D0661E0809112010E948D0661E08091AE
:1003D00010010E948D0661E080917E010E948D06D1
:1003E00061E080910E010E948D0661E080910C0118
:1003F0000E948D0661E080910A010E948D06809125
:100400007A0190917B01009711F460E004C0813083
:10041000910561F461E080917E010E94C60660E072
:1004200080910E010E94C60660E030C082309105C6
:1004300011F460E004C08330910539F461E08091EB
:100440007E010E94C60661E0EBCF8430910511F475
:1004500060E004C08530910539F461E080917E014F
:100460000E94C60660E00DC08630910511F460E080
:1004700003C0079779F461E080917E010E94C6066F
:1004800061E080910E010E94C60661E080910C013E
:100490000E94C60661E080911C010E94C60661E0D0
:1004A00080911A010E94C60660E0809112010C94AE
:1004B000C60640E855E260E070E080E891E00E9406
:1004C000E20761E0809122010E948D0660E0809148
:1004D00020010E948D060E94A90161E080910A011D
:1004E0000E94C60661E0809114010C94C60660E487
:1004F00071E082E791E00C948D0C82E791E00C941E
:100500001F0CCF93DF9380E891E00E944F07892B67
:1005100009F47DC280E891E00E945F078D3039F0D8
:10052000682F82E791E0DF91CF910C94E70C61E0B6
:10053000809122010E94C60688E893E190935F01B2
:1005400080935E0162E771E080E891E00E946908B3
:1005500060E070E082E791E00E94FA0CFC0180818B
:10056000803409F078C061E070E082E791E00E9499
:10057000FA0CFC0180818D3409F06DC062E070E0FE
:1005800082E791E00E94FA0CFC018081813409F03D
:1005900062C063E070E082E791E00E94FA0CFC0127
:1005A0008081823509F057C064E070E082E791E015
:1005B0000E94FA0CFC018081992787FD9095C097D5
:1005C00028EE33E0829FE001839FD00D929FD00DF3
:1005D000112465E070E082E791E00E94FA0CFC01D2
:1005E0008081992787FD9095C09744E6489F9001A8
:1005F000499F300D1124C20FD31F66E070E082E7DF
:1006000091E00E94FA0CFC018081992787FD90956A
:10061000C0974AE0489F9001499F300D1124C20FB6
:10062000D31F67E070E082E791E00E94FA0CFC01C2
:100630008081992787FD9095C0978C0F9D1F90937F
:1006400009018093080160E471E082E791E0DF91A5
:10065000CF910C94A30C60E070E082E791E00E94DF
:10066000FA0CFC018081803409F071C061E070E017
:1006700082E791E00E94FA0CFC0180818D3409F040
:1006800066C062E070E082E791E00E94FA0CFC0133
:100690008081813409F05BC063E070E082E791E023
:1006A0000E94FA0CFC018081833509F050C064E09F
:1006B00070E082E791E00E94FA0CFC0180819927AA
:1006C00087FD9095C09728EE33E0829FE001839FDD
:1006D000D00D929FD00D112465E070E082E791E08B
:1006E0000E94FA0CFC018081992787FD9095C097A4
:1006F00044E6489F9001499F300D1124C20FD31F3B
:1007000066E070E082E791E00E94FA0CFC018081D3
:10071000992787FD9095C0974AE0489F9001499F8F
:10072000300D1124C20FD31F67E070E082E791E023
:100730000E94FA0CFC018081992787FD9095C09753
:100740008C0F9D1F90930701809306017CCF60E082
:1007500070E082E791E00E94FA0CFC018081803415
:1007600009F075C061E070E082E791E00E94FA0C48
:10077000FC0180818D3409F06AC062E070E082E79C
:1007800091E00E94FA0CFC018081813409F05FC085
:1007900063E070E082E791E00E94FA0CFC01808146
:1007A000803509F054C064E070E082E791E00E9477
:1007B000FA0CFC018081992787FD9095C09728EE5F
:1007C00033E0829FE001839FD00D929FD00D1124D2
:1007D00065E070E082E791E00E94FA0CFC01808104
:1007E000992787FD9095C09744E6489F9001499FBF
:1007F000300D1124C20FD31F66E070E082E791E054
:100800000E94FA0CFC018081992787FD9095C09782
:100810004AE0489F9001499F300D1124C20FD31F19
:1008200067E070E082E791E00E94FA0CFC018081B1
:10083000992787FD9095C0978C0F9D1F20E031E090
:10084000281B390B3093710120937001FCCE60E0BE
:1008500070E082E791E00E94FA0CFC018081803414
:1008600051F461E070E082E791E00E94FA0CFC0133
:1008700080818D3461F060E070E082E791E00E9459
:10088000FA0CFC018081803409F0DDCE15C062E0F5
:1008900070E082E791E00E94FA0CFC0180818134D3
:1008A00051F763E070E082E791E00E94FA0CFC01EE
:1008B0008081813401F734C061E070E082E791E02B
:1008C0000E94FA0CFC0180818D3409F0BCCE62E0FC
:1008D00070E082E791E00E94FA0CFC018081813493
:1008E00009F0B1CE63E070E082E791E00E94FA0C7B
:1008F000FC018081883409F0A6CE81E090E09093DD
:100900006F0180936E019093650180936401109252
:100910006A0110926B0110926C0110926D0193CEDE
:100920008091640190916501892B09F067C064E0B2
:1009300070E082E791E00E94FA0CFC018081992727
:1009400087FD9095C09790936F0180936E0165E04D
:1009500070E082E791E00E94FA0CFC018081992707
:1009600087FD9095C09728EE33E0829FE001839F3A
:10097000D00D929FD00D112466E070E082E791E0E7
:100980000E94FA0CFC018081992787FD9095C09701
:1009900044E6489F9001499F300D1124C20FD31F98
:1009A00067E070E082E791E00E94FA0CFC01808130
:1009B000992787FD9095C0974AE0489F9001499FED
:1009C000300D1124C20FD31F68E070E082E791E080
:1009D0000E94FA0CFC018081992787FD9095C097B1
:1009E0008C0F9D1FAA2797FDA095BA2F80936A01AF
:1009F00090936B01A0936C01B0936D01109266010E
:100A00001092670110926801109269011CCEDF916B
:100A1000CF910895809120010E94FC069093790166
:100A2000809378010E94810280916E0190916F0104
:100A3000019711F461E001C060E0809114010E940F
:100A4000C6068091620190916301009709F07BC016
:100A50008091700190917101909363018093620184
:100A600040916A0150916B0160916C0170916D0130
:100A70008091660190916701A0916801B091690130
:100A800084179507A607B7073CF080916401909101
:100A90006501019709F04EC060910801709109014C
:100AA00080910A010E94B9058091600190916101D5
:100AB000019751F4109261011092600161E0809100
:100AC00010010E94C60644C08091640190916501A6
:100AD000019759F48091780190917901892B29F43B
:100AE000109265011092640133C060E080911001A2
:100AF0000E94C60681E090E09093610180936001BE
:100B00008091640190916501892B11F580916601B6
:100B100090916701A0916801B09169010196A11DB2
:100B2000B11D8093660190936701A0936801B09313
:100B300069010EC0609106017091070180910A0160
:100B40000E94B90505C001979093630180936201EB
:100B500080915E0190915F01009729F460E080919F
:100B600022010C94C606019790935F0180935E0169
:100B700008951F93CF93DF93182FEB0161E00E943C
:100B80008D06209711F460E004C0CF3FD10539F401
:100B900061E0812FDF91CF911F910C94C606E12F68
:100BA000F0E0E851FF4F449150E0FA013197EF3007
:100BB000F10508F06CC0EA5AFF4F0C943B0F84B566
:100BC000806884BDC7BD68C084B5806284BDC8BD6F
:100BD00063C080918000806880938000D0938900FA
:100BE000C093880059C0809180008062809380000B
:100BF000D0938B00C0938A004FC0809180008860A2
:100C000080938000D0938D00C0938C0045C080916C
:100C10009000806880939000D0939900C0939800D2
:100C20003BC080919000806280939000D0939B00A5
:100C3000C0939A0031C080919000886080939000AA
:100C4000D0939D00C0939C0027C08091C000806815
:100C50008093C0008091C0008F7B8093C000C093C0
:100C6000CF001AC08091C00080628093C000C09302
:100C7000D00012C08091C20088608093C200809131
:100C8000C2008B7F8093C200C093D20005C0C038E1
:100C9000D1050CF07DCF77CFDF91CF911F910895D3
:100CA00090E0FC013197EF30F105B0F5EB59FF4FC3
:100CB0000C943B0F809180008F7703C0809180005F
:100CC0008F7D80938000089580918000877FF9CF89
:100CD00084B58F7702C084B58F7D84BD08958091DF
:100CE00090008F7707C0809190008F7D03C0809126
:100CF0009000877F8093900008958091C0008F7747
:100D000003C08091C0008F7D8093C00008958091C2
:100D1000C200877F8093C2000895CF93DF9390E055
:100D2000FC01EA5FFE4F2491FC01EC5DFE4F8491D3
:100D3000882349F190E0880F991FFC01E25AFE4F89
:100D4000A591B491805B9E4FFC01C591D4919FB752
:100D5000611108C0F8948C91209582238C9388812E
:100D600082230AC0623051F4F8948C91322F30956E
:100D700083238C938881822B888304C0F8948C9180
:100D8000822B8C939FBFDF91CF9108950F931F9378
:100D9000CF93DF931F92CDB7DEB7282F30E0F90154
:100DA000E851FF4F8491F901EA5FFE4F1491F90178
:100DB000EC5DFE4F04910023C9F0882321F0698384
:100DC0000E9450066981E02FF0E0EE0FFF1FE05B0C
:100DD000FE4FA591B4919FB7F8948C91611103C017
:100DE0001095812301C0812B8C939FBF0F90DF91C1
:100DF000CF911F910F910895CF93DF93282F30E06B
:100E0000F901E851FF4F8491F901EA5FFE4FD49157
:100E1000F901EC5DFE4FC491CC2391F081110E9449
:100E20005006EC2FF0E0EE0FFF1FEE5BFE4FA5919A
:100E3000B4912C912D2381E090E021F480E002C058
:100E400080E090E0DF91CF910895CF93DF931F92E0
:100E5000CDB7DEB76983DC01ED91FC910280F381AF
:100E6000E02D41E050E0BE016F5F7F4F09950F908C
:100E7000DF91CF910895CF93DF93EC018C859D8511
:100E800097FF05C082E00E944C099D878C878C8566
:100E90009D85DF91CF91089583E00C94A10BFC0117
:100EA0008485958597FD06C082E00E94F40890E055
:100EB0000196089582E00E94F40890E00895FC01F4
:100EC0008485958597FD05C02FEF3FEF35872487F3
:100ED000089582E00C944C09CF93DF93EC0180914C
:100EE0002B01882331F083E00E947D091816190632
:100EF00034F081E090E09B838A8380E090E0DF9192
:100F0000CF910895FC0120812E5F208342E450E0C0
:100F10006CE671E080E80C94180AFC0181819081F4
:100F2000913A59F4813209F03CC047E050E064E264
:100F300071E080E00E94180A43C0913291F580323E
:100F400039F467E070E084E291E00E94490A06C04B
:100F5000823209F035C0828180932B018091240177
:100F600090912501A0912601B0912701803B9440EA
:100F7000A105B105C1F480912B0180FD14C087E764
:100F800097E790930108809300082BE088E190E0B8
:100F90000FB6F894A895809360000FBE2093600070
:100FA0000FC080E0089588E10FB6F8948093600048
:100FB000109260000FBEA8951092010810920008D0
:100FC00081E008952FEF3FEFFC01358724870895D6
:100FD000109283011092820188EE93E0A0E0B0E0CD
:100FE0008093840190938501A0938601B09387013B
:100FF00082E391E090938101809380018FEF9FEFD6
:1010000090938D0180938C01089508950E94A10D05
:101010000E94050880ED91E00E94010C0E94590297
:10102000C0E0D0E00E940A052097E1F30E94000092
:10103000F9CFCF92DF92EF92FF920F931F93CF934E
:10104000DF936C017A01EB01E60EF71E00E010E081
:10105000CE15DF0561F06991D601ED91FC9101900B
:10106000F081E02DC6010995080F191FF1CFC801C5
:10107000DF91CF911F910F91FF90EF90DF90CF9074
:1010800008956115710581F0DB010D900020E9F7ED
:10109000AD0141505109461B570BDC01ED91FC910C
:1010A0000280F381E02D099480E090E00895DC0156
:1010B000ED91FC91DB0114964D915C9115976D912A
:1010C0007C910280F381E02D09946EE371E00C9431
:1010D00041080F931F93CF93DF93EC010E945708B1
:1010E0008C01CE010E946508800F911FDF91CF9186
:1010F0001F910F9108954091D4015091D5012091F5
:10110000D2013091D30142175307B4F49091E80013
:101110009570E1F39091E80092FD19C08093F10081
:101120008091D4019091D50101968F739927892BD5
:1011300019F48EEF8093E8008091D4019091D5014D
:1011400001969093D5018093D40181E0089580E0C9
:101150000895CF92DF92FF920F931F93CF93DF9367
:101160001F92CDB7DEB7082F162F862F880F8E5F00
:1011700099830E947B0883E00E947B08F02EC02E9A
:101180009981D92E8C2D8F19811778F4F6018491CD
:101190000E947B08082F80E00E947B088023FFEFDD
:1011A000CF1ADF0A8111EECF01C081E00F90DF91ED
:1011B000CF911F910F91FF90DF90CF9008956150D4
:1011C00030F02091F100FC0120830196F8CF28989F
:1011D00084E68093D70108952FB7FC012083F8940B
:1011E00067706093E9000895CF93DF931F92CDB7A6
:1011F000DEB7682FCE0101960E94EC088091F200C4
:1012000099819FBF0F90DF91CF910895FF920F9327
:101210001F93CF93DF9300D0CDB7DEB7F62E8A01B0
:101220009091D601992311F057FF03C08FEF9FEFE4
:101230002BC0682FCE0101967A830E94EC08809122
:10124000F20090E0A8017A81801791070CF4AC01BC
:10125000EF2DF72FF40E84E6FE1639F028988093D0
:10126000D7019091F1009193F7CF4115510521F0ED
:101270008091F200882321F089818FBFCA0104C0C8
:101280008BE68093E800F8CF0F900F90DF91CF911D
:101290001F910F91FF900895CF93DF931F92CDB7C9
:1012A000DEB741E050E0BE016F5F7F4F0E9406094C
:1012B000019719F4898190E002C08FEF9FEF0F90A2
:1012C000DF91CF910895CF93DF931F92CDB7DEB713
:1012D000682FCE0101960E94EC089091E800892FBA
:1012E000807295FF04C09091F20080E4891B99817F
:1012F0009FBF0F90DF91CF9108956F927F928F9251
:101300009F92AF92BF92CF92DF92EF92FF920F9394
:101310001F93CF93DF931F92CDB7DEB7782E7B015B
:10132000C42EB52E8091D601882369F0042F152F85
:101330008AEFD82E872D8072982E9AE3A92E872DBA
:101340008074882E11C08FEF9FEF57C0872D0E94A9
:101350006309682E81110CC0DA94A9F361E070E092
:1013600080E090E00E94790D0115110579F73BC0EE
:10137000282F30E0021713070CF4602E672DCE01E2
:1013800001960E94EC088091E80085FF29C0262D77
:1013900030E0021B130B992039F06A948FEF681626
:1013A000B1F01092F100F9CFF701862D77FE07C05A
:1013B000815058F094919093F1003196F9CF81507B
:1013C00020F091919093F100FACFE20EF31E8091FC
:1013D000E80085FF0FC00115110511F481100AC046
:1013E00089818FBFC1CF5D9884E68093D8018C2D11
:1013F0009B2D03C0A092E800F3CF0F90DF91CF9117
:101400001F910F91FF90EF90DF90CF90BF90AF9022
:101410009F908F907F906F9008951092E9001092A6
:10142000D5011092D4019093D3018093D2010895F5
:10143000CF92DF92FF920F931F93CF93DF9300D051
:10144000CDB7DEB7F82E8A016B0101151105B1F099
:10145000F601F7FE02C0849101C0808149835A835E
:101460000E947B0801501109FFEFCF1ADF0A498162
:101470005A818111EACF8FEF9FEF01C0CA010F900F
:101480000F90DF91CF911F910F91FF90DF90CF9040
:1014900008951F93CF93DF931F92CDB7DEB7162F1A
:1014A0002091E80022FFFCCF612F79830E94DF08A2
:1014B0008BEF8093E800812F7981972F0F90DF9138
:1014C000CF911F910895CF93DF931F92CDB7DEB7D1
:1014D0001982CE0101960E948207CE0101960E94D8
:1014E000150E898190E00F90DF91CF9108951F92A2
:1014F0000F920FB60F921124EF92FF920F931F934A
:101500002F933F934F935F936F937F938F939F930B
:10151000AF93BF93EF93FF93CF93DF93CDB7DEB736
:101520006297DEBFCDBF1092E9008091E80083FF93
:10153000EBC068E0CE010A960E94DF0882EF80933C
:10154000E8009A8597FF05C08091E80080FFFCCFF6
:1015500003C08EEF8093E800892F807609F0B9C030
:101560008B85811105C01092F1001092F100C5C069
:10157000282F2D7F213009F4C0C0853049F4809197
:10158000E80080FFFCCF8C8580688093E300B5C0C5
:10159000863009F076C02D85E888F988223071F50B
:1015A00080E090E02A8B0E940D0A0E94630A99E075
:1015B0008E010F5F1F4FF801392F11923A95E9F70D
:1015C00099832A892A8391E09E8390E898879AEFED
:1015D00099872091D4013091D501275F3F4F3C83FB
:1015E0002B838D83C7010E940D0A49E050E0B801AA
:1015F00080E00E94180A0E94630A7FC0C7012A8BFC
:101600000E940D0A2A89223241F482E290E00E946F
:10161000200E892B09F071C074C0213069F48889CB
:101620009989089711F42093D1018091D1018111FA
:1016300018C065EC71E01AC0233009F062C08C85D7
:10164000882391F0823021F460E183EE91E006C0BE
:10165000813009F056C06BE087ED91E00E94A90847
:101660004AC063EB71E002C064EF71E0611571057F
:1016700009F447C0FB01449150E080E80E94180A39
:101680003CC0873009F43DC0883021F481E080936C
:10169000F10033C0893089F5937099F5EFEAF1E0F4
:1016A00081E021E096E38093E9002093EB00349100
:1016B0003093EC009093ED008F5F3196853099F771
:1016C0008EE78093EA001092EA008C858093D60121
:1016D00014C0888999890E940D0A8E85811105C0E0
:1016E000CE010A960E948D0706C0823051F4CE01C9
:1016F0000A960E94480E882321F08EEF8093E8001E
:1017000003C081E28093EB0062960FB6F894DEBFCF
:101710000FBECDBFDF91CF91FF91EF91BF91AF9100
:101720009F918F917F916F915F914F913F912F91F9
:101730001F910F91FF90EF900F900FBE0F901F9091
:1017400018958093E9008091F200882319F08AE3CC
:101750008093E80008951F920F920FB60F92112404
:101760002F933F934F935F936F937F938F939F93A9
:10177000AF93BF93EF93FF938091E1001092E1004C
:1017800083FF0FC01092E90091E09093EB0010925C
:10179000EC0092E39093ED001092D60198E09093C4
:1017A000F00082FF1DC083E00E94A10B8091D80150
:1017B000882339F08091D80181508093D801882303
:1017C00069F08091D701882359F08091D701815029
:1017D0008093D701811104C0289A02C05D9AF1CF8D
:1017E000FF91EF91BF91AF919F918F917F916F91F9
:1017F0005F914F913F912F910F900FBE0F901F90CF
:1018000018951092D60181E08093D70080EA8093EA
:10181000D80082E189BD09B400FEFDCF61E070E02F
:1018200080E090E00E94790D80E98093D8008CE000
:101830008093E2001092E000559A209A0895FC01EE
:10184000808191810C94D90FCF93DF93EC01888133
:101850009981009711F00E94D90F198218821D8278
:101860001C821B821A82DF91CF9108950F931F93E0
:10187000CF93DF93EC018B016F5F7F4F888199815C
:101880000E946810009731F0998388831B830A8334
:1018900081E001C080E0DF91CF911F910F91089509
:1018A000CF93DF93EC0188819981892B29F08A817C
:1018B0009B818617970760F4CE010E94360C88231F
:1018C00041F08C819D81892B19F4E881F981108286
:1018D00081E0DF91CF910895EF92FF920F931F93D4
:1018E000CF93DF93EC017B018A01BA010E94500C77
:1018F000811104C0CE010E94240C07C01D830C83FB
:10190000B701888199810E943B11CE01DF91CF916F
:101910001F910F91FF90EF900895FC0111821082AA
:1019200013821282158214826115710559F0FB0130
:1019300001900020E9F7AF0141505109461B570BB8
:101940000C946C0C0895CF93DF93EC016115710535
:1019500061F0FB0101900020E9F7AF01415051090E
:10196000461B570B0E946C0C02C00E94240CCE0137
:10197000DF91CF910895EF92FF920F931F93CF9332
:10198000DF93EC017B010C811D816115710511F460
:1019900080E016C04115510591F0040F151FB801E4
:1019A0000E94500C8823A1F3288139818C819D816C
:1019B000B701820F931F0E943B111D830C8381E0AE
:1019C000DF91CF911F910F91FF90EF900895CF93EA
:1019D000DF9300D0CDB7DEB769831A8241E050E0D3
:1019E000BE016F5F7F4F0E94BB0C0F900F90DF9185
:1019F000CF910895FC01848195816817790720F4BF
:101A000080819181009729F41092D90189ED91E0AC
:101A10000895860F971F08951F920F920FB60F9289
:101A200011242F933F938F939F93AF93BF938091F4
:101A3000DB019091DC01A091DD01B091DE013091DC
:101A4000DA0123E0230F2D3720F40196A11DB11DEB
:101A500005C026E8230F0296A11DB11D2093DA01CF
:101A60008093DB019093DC01A093DD01B093DE0154
:101A70008091DF019091E001A091E101B091E2013C
:101A80000196A11DB11D8093DF019093E001A09309
:101A9000E101B093E201BF91AF919F918F913F918E
:101AA0002F910F900FBE0F901F9018953FB7F8948D
:101AB0008091DF019091E001A091E101B091E201FC
:101AC00026B5A89B05C02F3F19F00196A11DB11D99
:101AD0003FBF6627782F892F9A2F620F711D811DB6
:101AE000911D42E0660F771F881F991F4A95D1F715
:101AF0000895CF92DF92EF92FF92CF93DF936B0125
:101B00007C010E94560DEB01C114D104E104F104E3
:101B100089F00E943A0F0E94560D6C1B7D0B683EA7
:101B2000734090F381E0C81AD108E108F108C85168
:101B3000DC4FEACFDF91CF91FF90EF90DF90CF9015
:101B40000895789484B5826084BD84B5816084BD35
:101B500085B5826085BD85B5816085BDEEE6F0E026
:101B6000808181608083E1E8F0E010828081826082
:101B70008083808181608083E0E8F0E08081816003
:101B80008083E1E9F0E080818260808380818160F0
:101B90008083E0E9F0E0808181608083E1ECF0E027
:101BA0008081846080838081826080838081816085
:101BB0008083E3ECF0E0808181608083E0ECF0E002
:101BC000808182608083E2ECF0E0808181608083AC
:101BD000EAE7F0E080818460808380818260808396
:101BE0008081816080838081806880830895FF92F6
:101BF0000F931F93CF93DF93EC01F62EE881F981C9
:101C00000480F581E02D09958C01E881F981068039
:101C1000F781E02D6F2DCE010995C8019927DF913D
:101C2000CF911F910F91FF900895FC0120812F5FAC
:101C3000208349E150E068E772E080E80C94180ADC
:101C400045E650E061E972E080E80C94180AEF92F2
:101C5000FF920F931F93CF93DF931F92CDB7DEB701
:101C600089838B017A0141E050E0BE016F5F7F4FB5
:101C700084E00E947D09A701B80184E40E947D09E7
:101C80000F90DF91CF911F910F91FF90EF900895EA
:101C9000FC0191818081813A31F481E0913091F0B1
:101CA000933089F411C0813271F49B3021F4828128
:101CB00080932D0105C09A3031F4828180932C01EC
:101CC00081E00895089580E0089548E050E082E0C2
:101CD0000C94270ECF93DF93DC01683818F0E8E707
:101CE000E60F25C0E62FF0E067FF11C0E058F109CC
:101CF00081E090E001C0880FEA95EAF714969C9184
:101D00001497982B14969C931497E0E010C0E85019
:101D1000FE4FE491EE2309F440C0E7FF08C014969B
:101D20008C911497826014968C931497EF77169683
:101D30008C9116978E1741F117968C9117978E17E5
:101D400019F118968C9118978E17F1F019968C91BD
:101D500019978E17C9F01A968C911A978E17A1F0C1
:101D60001B968C911B978E1779F080E090E0ED0127
:101D7000C80FD91F2E81211102C0EE8305C0019624
:101D800086309105A1F709C0BD016C5F7F4FCD0181
:101D90000E94650E81E090E008C081E090E013961B
:101DA0009C938E93129780E090E0DF91CF910895FD
:101DB000683818F0E8E7E60F25C0E62FF0E067FF87
:101DC00012C0E058F10921E030E001C0220FEA958D
:101DD000EAF72095DC0114963C911497322314966F
:101DE0003C93E0E00FC0E850FE4FE491EE2329F170
:101DF000E7FF08C0DC0114962C9114972D7F1496F0
:101E00002C93EF7720E030E0EE2351F0DC01A20FBD
:101E1000B31F16964C9116974E1302C016961C923D
:101E20002F5F3F4F2630310579F7BC016C5F7F4F44
:101E30000E94650E81E090E0089580E090E00895B2
:101E4000FC01168217821086118612861386148270
:101E5000BC016C5F7F4F0C94650E1092EF011092E5
:101E6000E6011092E50183E591E09093E40180930F
:101E7000E30108950895EE0FFF1F0590F491E02D02
:101E80000994CF93DF938230910510F482E090E0C3
:101E9000E091F201F091F30120E030E0A0E0B0E049
:101EA000309739F14081518148175907B8F04817E8
:101EB000590771F482819381109729F013969C93AE
:101EC0008E9312972CC09093F3018093F20127C058
:101ED0002115310531F04217530718F0A901DB0134
:101EE00001C0EF019A01BD01DF010280F381E02D05
:101EF000D7CF21153105F9F0281B390B24303105D6
:101F000080F48A819B816115710521F0FB01938327
:101F1000828304C09093F3018093F201FE01329614
:101F200044C0FE01E20FF31F8193919322503109C7
:101F3000398328833AC02091F0013091F101232B9D
:101F400041F420910201309103013093F10120937B
:101F5000F00120910001309101012115310541F47A
:101F60002DB73EB74091040150910501241B350B5C
:101F7000E091F001F091F101E217F307A0F42E1BBC
:101F80003F0B2817390778F0AC014E5F5F4F2417DD
:101F9000350748F04E0F5F1F5093F1014093F00159
:101FA0008193919302C0E0E0F0E0CF01DF91CF9107
:101FB0000895CF93DF93009709F487C0FC0132970F
:101FC00013821282C091F201D091F301209781F423
:101FD00020813181280F391F8091F0019091F1010A
:101FE0008217930779F5F093F101E093F0016DC04A
:101FF000DE0120E030E0AE17BF0750F412964D919D
:102000005C9113979D014115510509F1DA01F3CF58
:10201000B383A28340815181840F951F8A179B0748
:1020200071F48D919C911197840F951F0296918365
:10203000808312968D919C911397938382832115AF
:10204000310529F4F093F301E093F2013EC0D90188
:102050001396FC93EE9312974D915D91A40FB51FCB
:10206000EA17FB0779F480819181840F951F02960E
:10207000D90111969C938E938281938113969C93A0
:102080008E931297E0E0F0E08A819B81009719F02F
:10209000FE01EC01F9CFCE01029628813981820F31
:1020A000931F2091F0013091F1012817390769F44D
:1020B000309729F41092F3011092F20102C01382BA
:1020C0001282D093F101C093F001DF91CF91089576
:1020D000A0E0B0E0EEE6F0E10C944611EC01CB019B
:1020E000209719F40E94410FB8C0FE01E60FF71FB8
:1020F0009E0122503109E217F30708F4ACC0D90160
:102100000D911C91119706171707B8F005301105AE
:1021100008F49FC0A801445051094617570708F416
:1021200098C002501109061B170B019311936D9370
:102130007C93CF010E94D90F8CC05B01A01AB10A19
:102140004E01800E911EA091F201B091F301612C1D
:10215000712C60E070E0109709F449C0A815B9052A
:10216000C9F5ED90FC901197670142E0C40ED11CB7
:10217000CA14DB0478F147018A189B08640142E025
:10218000C40ED11C1296BC9012971396AC91B5E078
:10219000CB16D10440F0B282A38391828082D90110
:1021A0008D939C9309C00E5F1F4F0E0D1F1DF901EB
:1021B00011830083EB2DFA2F6115710531F0DB01DE
:1021C0001396FC93EE93129744C0F093F301E093BF
:1021D000F2013FC06D917C9111976616770608F465
:1021E0003B01BD0112960D90BC91A02DB4CF609122
:1021F000F0017091F10168157905E9F46816790626
:10220000D0F440910001509101014115510541F474
:102210004DB75EB76091040170910501461B570BE5
:10222000E417F507C0F4F093F101E093F001F90130
:10223000918380830EC00E94410F7C01009759F06A
:10224000A801BE010E943211CE010E94D90FC70120
:1022500004C0CE0102C080E090E0CDB7DEB7EEE072
:102260000C946211FB01DC0102C001900D924150FF
:102270005040D8F70895FB01DC0101900D92002039
:10228000E1F708952F923F924F925F926F927F9263
:102290008F929F92AF92BF92CF92DF92EF92FF9276
:1022A0000F931F93CF93DF93CDB7DEB7CA1BDB0B22
:1022B0000FB6F894DEBF0FBECDBF09942A883988C7
:1022C00048885F846E847D848C849B84AA84B984CE
:1022D000C884DF80EE80FD800C811B81AA81B981DA
:1022E000CE0FD11D0FB6F894DEBF0FBECDBFED01EE
:1022F000089512E0CCEFD2E004C0FE010E943D0F31
:0C2300002296CE3FD107C9F7F894FFCF1A
:10230C000000F40180008000FF00050003000200C3
:10231C00010004000C000600080009000A000B0074
:10232C0007000D0000E100000000000001010000AA
:10233C00000025076C074F075F073B074C070D0A8A
:10234C00006E616E00696E66006F7666002E00008E
:0E235C00000000F70D19086A0ED80E200F00C1
:00000001FF
